:020000040000FA
:02000000A42832
:080008001728A801A701260832
:10001000A900A70B0928A80B0928A90B0928080083
:100020000C1299008316981C1328831208008C1E4A
:1000300009008B138C121A08A000513020020319FA
:10004000452857302002031948284530200203195B
:100050004B28523020020319522854302002031931
:10006000562859302002031940284930200203192C
:100070005B280B178B17200810200D30102009006B
:100080002A110708F939870039282A152A10392832
:100090002A152A143928AA1C4E285028AA143928AF
:1000A000AA103928A60B3928A60A3928A60F3928FC
:1000B000FF30A60039288316FF308600831205081A
:1000C000A1000608A2000708A3000808A400093040
:1000D00010208F208C2089208620832080207D2066
:1000E0007A20203010209220952098209B200930E3
:1000F00010203928A21FA1289E28221FA1289E284F
:10010000A21EA1289E28221EA1289E28A21DA12849
:100110009E28221DA1289E28A21CA1289E28221CC0
:10012000A1289E28241FA1289E28A41FA1289E281C
:10013000211EA1289E28231CA1289E283030102093
:1001400008003130102008008316FF308500FF3092
:10015000860099308700C0308800890124309800DB
:10016000403099008C1683128701880189019030F4
:1001700098000B178B170130A6002A1DBD28AA1C5A
:10018000BD282A18C728AB030330AB05CA28AB0A21
:100190000330AB052B08D2208800070806388700FB
:0E01A0000520BD2882070234003401340334E8
:02400E003A3F37
:00000001FF
